:10000000E9EF02F00000000000EF00F00000000047
:0A0010000000000000000000F3D71C
:10001C00240E0C6EB50E0D6E0D2EFED70C2EFCD7CD
:06002C00000000001200BC
:0A003200530E0D6E0D2EFED71200C6
:0C003C00000000000000000000001200A6
:10004800010124BF02D08A9A01D08A8A24BD02D035
:100058008A9801D08A8824BB02D08A9601D08A86E1
:1000680024B902D08A9401D08A8400016FB102D0E9
:100078008A8001D08A908A82DDDF8A92010124B7C2
:1000880002D08A9A01D08A8A24B502D08A9801D0EF
:100098008A8824B302D08A9601D08A8624B102D0F5
:1000A8008A9401D08A8400016FB102D08A8001D07D
:1000B8008A908A82BFDF8A926FA102D0ABDF01D01B
:0400C800B4DF12008F
:1000CC00AECF02F0ABA202D0AB98AB8802C001F06D
:0600DC0001C000F012005B
:1000E200086A080E0C6E003408360450085ED8B058
:0E00F20002D00826D89000360C2EF5D712004A
:0E01000000016F9121C124F19FDF6F81120079
:0E010E00000E9EBA010E016E01C000F012003C
:10011C0001012151010A03E1800E216F14D02151FC
:10012C00020A03E1C00E216F0ED02151030A03E134
:10013C00940E216F08D02151040A03E1D40E216FD3
:10014C0002D0800E216F2205006E2151002600C0C6
:10015C0021F100016F8100C024F170DF6F9123C188
:08016C0024F16CDF6F81120029
:10017400016A015001011D5D18E301501E25E16E65
:10018400000E1F21E26E01501C25006EC00EE96EA8
:10019400000EEA6E0050E926D8B0EA2AEECFE6FF58
:1001A40001501D1902E0012AE4D71D511E25E16EFC
:0C01B400000E1F21E26E000EE66E12002D
:1001C0001DC1E1FF1EC1E2FF200EE66E200EE66EAD
:1001D000300EE66EE66A020E01011D251F6F000E4D
:1001E0001E21206F1C51000A1AE00A0E046E1CC169
:1001F00000F077DF08C000F01FC1E1FF20C1E2FF7F
:10020000300E0024E66E0A0E046E1CC100F069DF99
:1002100000C01CF1010E1F5F000E205BE3D712002F
:10022000700E0101246F10DF01011E6BB80E1E2538
:10023000F66E110EF76E000EF722000EF86E000E2D
:10024000F8220900F5CF21F15BDF01011E51070AF9
:1002500002E01E2BEBD7020E246FF6DE1CC121F14B
:0E0260001DC122F1060E0101236F58DF1200AE
:10026E000900F5CFE6FF0006FBE10106F9E11200F9
:10027E00500E0101246FE1DE01011E6BB00E1E2532
:10028E00F66E110EF76E000EF722000EF86E000ECF
:10029E00F8220900F5CF21F12CDF01011E51070ACA
:1002AE0002E01E2BEBD7020E246FC7DE1CC121F11C
:0E02BE001DC122F1020E0101236F29DF120083
:1002CC0001011C51010A03E1800E1C6F14D01C515A
:1002DC00020A03E1C00E1C6F0ED01C51030A03E18D
:1002EC00940E1C6F08D01C51040A03E1D40E1C6F31
:1002FC0002D0800E1C6F1D05006E1C51002600C024
:10030C001CF100C024F19ADE6F910101206B205189
:10031C001E25E96E000E1F21EA6EEE50000A0CE05D
:10032C0020511E25E96E000E1F21EA6EEECF21F141
:0E033C00E1DE0101202BEBD700016F811200E2
:10034A00FF0E00016B6FFF0E6C6FFF0E6D6FFF0EDD
:10035A006E6FCC0E786F000E796F000E7A6F000EFA
:10036A007B6F0E0E746F010E756F000E766F000EA6
:10037A00776FFF0E706FFF0E716F000E726F000EB7
:10038A00736FAC8A900EAB6E948E949C9EAA03D027
:08039A00AECF00F0FBD712000A
:1003A20093929390939493969398939A8A928A9025
:1003B2008A9A8A988A968A9430DE2FDE2EDE8A8680
:1003C2008A848A823ADE8A9228DE8A8236DE8A929B
:1003D20024DE8A8232DE8A9220DE8A948A822DDEAE
:1003E2008A921BDE8A8229DE8A928A968A8A8A8287
:1003F20024DE8A9212DE8A9A8A848A821EDE8A9297
:100402008A948A821ADE8A9208DE8A8216DE8A92AA
:100412008A848A8212DE8A9200DE8A948A820DDEC1
:100422008A928A8A8A888A868A848A8206DE8A925E
:08043200F4DD00016F811200EE
:10043A00480E0101246F03DE01011E6BA80E1E2562
:10044A00F66E110EF76E000EF722000EF86E000E11
:10045A00F8220900F5CF21F14EDE01011E51070AEB
:10046A0002E01E2BEBD7020E246FE9DD1CC121F13D
:0E047A001DC122F1010E0101236F4BDE1200A5
:10048800400E0101246FDCDD01011E6B980E1E2554
:10049800F66E110EF76E000EF722000EF86E000EC3
:1004A800F8220900F5CF21F127DE01011E51070AC4
:1004B80002E01E2BEBD7020E246FC2DD1CC121F116
:0C04C8001DC122F10101236B25DE120092
:1004D400680E0101246FB6DD01011E6B900E1E250E
:1004E400F66E110EF76E000EF722000EF86E000E77
:1004F400F8220900F5CF21F101DE01011E51070A9E
:1005040002E01E2BEBD7020E246F9CDD1CC121F1EF
:0E0514001DC122F1050E0101236FFEDD120054
:10052200F5DD0050010AFCE1D0DD00C01CF11CC168
:0405320000F01200C3
:10053600580E0101246F85DD01011E6B880E1E25F4
:10054600F66E110EF76E000EF722000EF86E000E14
:10055600F8220900F5CF21F1D0DD01011E51070A6D
:1005660002E01E2BEBD7020E246F6BDD1CC121F1BE
:0E0576001DC122F1030E0101236FCDDD120025
:10058400600E0101246F5EDD01011E6BA00E1E25AD
:10059400F66E110EF76E000EF722000EF86E000EC6
:1005A400F8220900F5CF21F1A9DD01011E51070A46
:1005B40002E01E2BEBD7020E246F44DD1CC121F197
:0E05C4001DC122F1040E0101236FA6DD1200FD
:1005D200B886020EB06E080EAF6EAC84B5DE030EA6
:1005E2000B6E8A0E0C6E550E0D6E0D2EFED70C2E56
:1005F200FCD70B2EFAD700000000929494809482CC
:10060200CFDE010E0101246F1EDD0C0E0101246FED
:100612001ADD8984010E01011C6F010E1D6F200E6F
:10062200056F200E066F200E076F520E086F450EE3
:10063200096F430E0A6F450E0B6F500E0C6F540E6E
:100642000D6F450E0E6F550E0F6F520E106F200E6E
:10065200116F470E126F500E136F530E146F200E50
:10066200156F200E166F200E176F200E186F196B64
:10067200050E1E6F010E1F6F28DE020E01011C6F98
:10068200010E1D6F4D0E056F4F0E066F440E076F64
:10069200550E086F4C0E096F450E0A6F200E0B6F38
:1006A200520E0C6F450E0D6F590E0E6F410E0F6FED
:1006B200580E106F200E116F520E126F470E136FED
:1006C200320E146F350E156F440E166F490E176FEA
:1006D200200E186F196B050E1E6F010E1F6FF5DDD0
:1006E200040E01011C6F010E1D6F490E056F6E0E87
:1006F200066F690E076F740E086F690E096F610E3F
:100702000A6F6C0E0B6F690E0C6F730E0D6F610E1C
:100712000E6F740E0F6F690E106F6F0E116F6E0EEB
:10072200126F2E0E136F2E0E146F2E0E156F2E0ECD
:10073200166F2E0E176F186B050E1E6F010E1F6FB0
:10074200C4DD660E0B6E760E0C6EC10E0D6E0D2E96
:10075200FED70C2EFCD70B2EFAD7010E0101046F27
:10076200560E036F0001BF6B010E5D6E300E526EAE
:10077200300E536E546A516A82A203D02F0E5F6EFE
:1007820002D02E0E5F6ECCDE00C05EF00050240A56
:1007920001E0F9D75E6AC00E01011A6F000E1B6FED
:1007A2005E501A27D8B01B2BBBDE1AC1E1FF1BC15A
:1007B200E2FF00C0E6FFC00EE96E000EEA6E5E5078
:1007C200E926D8B0EA2AEE502A0A02E15E6A01D08E
:1007D2005E2A5E50000AFF0ED8A4000E016E5E5023
:1007E200420AFF0ED8A4000E006E0150001201E171
:1007F200D2D701010451010AD8A499D00001C251F3
:10080200520AFF0ED8A4000E016EC3514D0AFF0E0C
:10081200D8A4000E006E00500116C451430AFF0E08
:10082200D8A4000E006E01500016D8B480D0020E7B
:100832000101046F010E0001BF6F03C15EF0D0C061
:1008420003F1D0515E1805E0010E0101246F24EC82
:1008520000F001010351410A6AE18984060E1C6F0E
:10086200060E1D6F460E1E6F000E1F6F82DC300ECD
:10087200465C006E0A0E0002F3CF00F047500026DD
:100882005F50005E00C05EF000C01CF12B0E1D6FB9
:10089200000E1E6F94DC120E1C6F020E1D6F200ED6
:1008A2001E6F000E1F6F65DC140E1C6F020E1D6F93
:1008B200150E1E6F000E1F6F5CDC170E1C6F050EEF
:1008C2001D6F3B0E1E6F000E1F6F53DCDDC03AF032
:1008D2001F0E1C6F030E1D6F2F0E1E6F000E1F6F5B
:1008E20048DC220E1C6F020E1D6F600E1E6F000E82
:1008F2001F6F3FDC250E1C6F050E1D6F930E1E6FC2
:10090200000E1F6F36DCEBC092F02D0E1C6F040E32
:100912001D6F870E1E6F000E1F6F2BDC340E1C6FB7
:10092200060E1D6FB40E1E6F000E1F6F22DC01013A
:100932000451020A4BE10001C251470AFF0ED8A43A
:10094200000E016EC351470AFF0ED8A4000E006EBE
:1009520000500116C451410AFF0ED8A4000E006EC9
:100962000150001633E0010E0101046F010E000177
:10097200BF6F01010351410A29E189842D0E1C6FC9
:10098200020E1D6F520E1E6F000E1F6FBAEC00F0AA
:10099200300E1C6F040E1D6FA90E1E6F000E1F6F0E
:1009A200BAEC00F0350E1C6F050E1D6F9E0E1E6F09
:1009B200000E1F6FBAEC00F03D0E1C6F040E1D6F8F
:1009C2007C0E1E6F000E1F6FBAEC00F00001BF51CB
:1009D200010AD8A4D5D382A003D0010E5D6E02D045
:1009E200020E5D6E01010351560AD8A4DBD0899430
:1009F200010E1C6F010E1D6F200E056F200E066F7B
:100A0200200E076F200E086F200E096F450E0A6F29
:100A12004E0E0B6F200E0C6F410E0D6F540E0E6FAB
:100A2200540E0F6F450E106F4E0E116F540E126F53
:100A3200450E136F200E146F200E156F200E166FC9
:100A4200200E176F200E186F196B050E1E6F010E08
:100A52001F6F3BDC020E01011C6F010E1D6F200E89
:100A6200056F200E066F200E076F200E086F200EF6
:100A7200096F200E0A6F200E0B6F200E0C6F200ED6
:100A82000D6F440E0E6F450E0F6F200E106F200E6D
:100A9200116F200E126F200E136F200E146F200E96
:100AA200156F200E166F200E176F200E186F196B20
:100AB200050E1E6F010E1F6F08DC030E01011C6F75
:100AC200010E1D6F200E056F200E066F200E076FA0
:100AD200540E086F520E096F410E0A6F4D0E0B6FC6
:100AE200450E0C6F530E0D6F200E0E6F560E0F6FCC
:100AF200410E106F4C0E116F490E126F440E136FA0
:100B0200450E146F530E156F200E166F200E176FC1
:100B1200200E186F196B050E1E6F010E1F6F66EC0B
:100B220001F0040E01011C6F010E1D6F200E056FF6
:100B3200200E066F200E076F200E086F200E096F21
:100B4200200E0A6F200E0B6F200E0C6F200E0D6F01
:100B5200200E0E6F200E0F6F200E106F200E116FE1
:100B6200200E126F200E136F200E146F200E156FC1
:100B7200200E166F200E176F200E186F196B050EC0
:100B82001E6F010E1F6F66EC01F0512A040E010167
:100B92001C6F51C01DF110EC01F05150140AD8B471
:100BA200516AECD25D50010AD8A4B8D1010E0101FC
:100BB2001C6F010E1D6F4C0E056F610E066F740ED9
:100BC200076F200E086F3A0E096F200E0A6F200E73
:100BD2000B6F0C6B050E1E6F010E1F6F66EC01F0A2
:100BE200010E01011C6F080E1D6F200E1E6F000EFC
:100BF2001F6F66EC01F0010E0101216F0A0E226FD8
:100C0200DF0E236F8EEC00F0010E01011C6F0B0E44
:100C12001D6F150E1E6F000E1F6F66EC01F0010EA8
:100C22000101216F0D0E226F2E0E236F8EEC00F04C
:100C3200010E01011C6F0E0E1D6F3B0E1E6F000E8A
:100C42001F6F66EC01F0010E0101216F130E226F7E
:100C5200200E236F8EEC00F0010E0101216F140EA5
:100C6200226F3AC023F18EEC00F0020E01011C6FDC
:100C7200010E1D6F4C0E056F6F0E066F6E0E076F25
:100C8200200E086F3A0E096F200E0A6F0B6B050ECD
:100C92001E6F010E1F6F66EC01F0020E01011C6F48
:100CA200070E1D6F2F0E1E6F000E1F6F66EC01F0F8
:100CB200020E0101216F0A0E226FDF0E236F8EECEE
:100CC20000F0020E01011C6F0B0E1D6F600E1E6FF5
:100CD200000E1F6F66EC01F0020E0101216F0D0E76
:100CE200226F2E0E236F8EEC00F0020E01011C6F9C
:100CF2000E0E1D6F930E1E6F000E1F6F66EC01F03D
:100D0200020E0101216F130E226F200E236F8EEC53
:100D120000F0020E0101216F140E226F92C023F126
:100D22008EEC00F0030E01011C6F010E1D6F410ECF
:100D3200056F6C0E066F740E076F200E086F3A0E69
:100D4200096F200E0A6F0B6B050E1E6F010E1F6FCF
:100D520066EC01F0030E01011C6F070E1D6F9E0E63
:100D62001E6F000E1F6F66EC01F0030E01011C6F77
:100D72000A0E1D6F6AEC02F0030E01011C6F0C0ECD
:100D82001D6F200E056F6D0E066F650E076F740ED8
:100D9200086F720E096F650E0A6F730E0B6F200ECD
:100DA2000C6F200E0D6F0E6B050E1E6F010E1F6F66
:100DB20066EC01F0030E01011C6F0E0E1D6F44EC78
:100DC20002F0040E0101216F010E226FB4C023F163
:100DD2008EEC00F0040E0101216F020E226FB5C0ED
:100DE20023F18EEC00F0040E01011C6F030E1D6F47
:100DF200C2EC02F0040E0101216F040E226FB6C094
:100E020023F18EEC00F0040E0101216F050E226F1A
:100E1200B7C023F18EEC00F0040E01011C6F060E28
:100E22001D6FC2EC02F0040E01011C6F070E1D6F54
:100E3200320E056F300E066F076B050E1E6F010E28
:100E42001F6F66EC01F0040E0101216F090E226F83
:100E5200B8C023F18EEC00F0040E0101216F0A0EDE
:100E6200226FB9C023F18EEC00F0040E01011C6F59
:100E72000B0E1D6F200E056F200E066F076B050E01
:100E82001E6F010E1F6F66EC01F0040E0101216F4F
:100E92000D0E226F2CC023F18EEC00F0040E010126
:100EA200216F0E0E226F2DC023F18EEC00F0040E86
:100EB2000101216F0F0E226F3A0E236F8EEC00F0AC
:100EC200040E0101216F100E226F48C023F18EEC37
:100ED20000F0040E0101216F110E226F49C023F1AF
:100EE2008EEC00F0040E0101216F120E226F3A0EF9
:100EF200236F8EEC00F0040E0101216F130E226F9E
:100F02004AC023F18EEC00F0040E0101216F140E91
:100F1200226F4BC023F18EEC00F030D15D50020AFB
:100F2200D8A42CD1010E01011C6F010E1D6F200EE1
:100F3200056F4E0E066F4D0E076F450E086F410E80
:100F4200096F200E0A6F300E0B6F310E0C6F380EC8
:100F52000D6F330E0E6F200E0F6F390E106F360E9F
:100F6200116F300E126F300E136F200E146F380E89
:100F7200156F4E0E166F310E176F200E186F196B0C
:100F8200050E1E6F010E1F6F66EC01F0020E0101CD
:100F92001C6F010E1D6F4E0E056F620E066F720EF4
:100FA200076F650E086F200E096F640E0A6F650EDB
:100FB2000B6F200E0C6F730E0D6F610E0E6F740EA1
:100FC2000F6F2E0E106F3A0E116F200E126F136BF1
:100FD200050E1E6F010E1F6F66EC01F0020E01017D
:100FE2001C6F0F0E1D6F520E1E6F000E1F6F66ECF0
:100FF20001F0020E01011C6F110E1D6F200E056F14
:10100200200E066F200E076F200E086F096B050E6B
:101012001E6F010E1F6F66EC01F0030E01011C6FC3
:10102200010E1D6F480E056F440E066F4F0E076FBF
:10103200500E086F3A0E096F200E0A6F0B6B050EE9
:101042001E6F010E1F6F66EC01F0030E01011C6F93
:10105200070E1D6FA90E1E6F000E1F6F66EC01F0CA
:10106200030E01011C6F080E1D6F6AEC02F0030EE5
:1010720001011C6F0B0E1D6F200E056F200E066FF7
:10108200200E076F200E086F200E096F200E0A6FC8
:10109200200E0B6F200E0C6F200E0D6F200E0E6FA8
:1010A2000F6B050E1E6F010E1F6F66EC01F0040E32
:1010B20001011C6F010E1D6F450E056F630E066F59
:1010C200610E076F720E086F740E096F2D0E0A6F94
:1010D200670E0B6F650E0C6F6F0E0D6F690E0E6F44
:1010E200640E0F6F650E106F3A0E116F200E126FA5
:1010F200136B050E1E6F010E1F6F66EC01F0040EDE
:1011020001011C6F060E1D6FC2EC02F0040E0101FC
:101112001C6F070E1D6F9BEC02F0040E01011C6F89
:10112200080E1D6F1DEC02F0040E01011C6F0A0E69
:101132001D6F3FEC01F0040E01011C6F0F0E1D6FBD
:101142007C0E1E6F000E1F6F66EC01F0040E010193
:101152001C6F110E1D6F6AEC02F0040E01011C6F70
:10116200130E1D6F200E056F6D0E066F076B050EB9
:101172001E6F010E1F6F66EC01F000D00001BF6B05
:06118200BDEF03F0FFD7F2
:0811880000000F11110F010E10
:0811900000000000000C04083F
:0811980008040E111F100E00E7
:0811A0000000000E0000000039
:0811A80002040E111F100E00DD
:0811B0000A0004040404040019
:0811B800181C1E1F1F1E1C184D
:020000040030CA
:0E000000000C1F1EFF8381FF0FC00FE00F409A
:00000001FF
